:020000040000FA
:0408000063EF09F0A9
:1008100003B283EF05F0F2B4A1EF05F09EB0A9EFAB
:1008200005F09EB2B1EF05F0F2A81AEF04F0F2B2B3
:1008300032EF04F09EB61FEF04F012EF09F09E961F
:1008400000011350000A06E000011350010A06E0FF
:1008500012EF09F009EC1FF012EF09F0FDEC20F0A7
:1008600012EF09F0CD90F2929EA03CEF04F001014E
:10087000533F3CEF04F0542BAEC1B2F1AFC1B3F122
:10088000B0C1B4F1B1C1B5F1AAC1AEF1ABC1AFF124
:10089000ACC1B0F1ADC1B1F1A6C1AAF1A7C1ABF134
:1008A000A8C1ACF1A9C1ADF1A2C1A6F1A3C1A7F144
:1008B000A4C1A8F1A5C1A9F19EC1A2F19FC1A3F154
:1008C000A0C1A4F1A1C1A5F19AC19EF19BC19FF164
:1008D0009CC1A0F19DC1A1F196C19AF197C19BF174
:1008E00098C19CF199C19DF1CECF96F1CFCF97F1F0
:1008F00053C198F154C199F1CF6ACE6A0101536B8B
:10090000546B9E90CD800FBC0F8E0FBA8BEF04F00E
:100910000F8A12EF09F00F8C0FBEC7EF04F096C1DB
:100920009AF197C19BF198C19CF199C19DF19AC12F
:100930009EF19BC19FF19CC1A0F19DC1A1F19EC1FF
:10094000A2F19FC1A3F1A0C1A4F1A1C1A5F1A2C1CF
:10095000A6F1A3C1A7F1A4C1A8F1A5C1A9F1A6C19F
:10096000AAF1A7C1ABF1A8C1ACF1A9C1ADF1AAC16F
:10097000AEF1ABC1AFF1ACC1B0F1ADC1B1F1AEC13F
:10098000B2F1AFC1B3F1B0C1B4F1B1C1B5F1010180
:100990005E6B5F6B606B616B96515E2797515F2357
:1009A00098516023995161239A515E279B515F238F
:1009B0009C5160239D5161239E515E279F515F236F
:1009C000A0516023A1516123A2515E27A3515F234F
:1009D000A4516023A5516123A6515E27A7515F232F
:1009E000A8516023A9516123AA515E27AB515F230F
:1009F000AC516023AD516123AE515E27AF515F23EF
:100A0000B0516023B1516123B2515E27B3515F23CE
:100A1000B4516023B5516123D89001016133603333
:100A20005F335E33D8900101613360335F335E33EF
:100A3000D8900101613360335F335E3300C10CF144
:100A400001C10DF102C10EF103C10FF104C110F19A
:100A500005C111F106C112F107C113F108C114F16A
:100A600009C115F10AC116F10BC117F134C135F1F5
:100A700011B846EF05F00101620E046F010E056F1B
:100A8000000E066F000E076F4FEF05F00101A70E75
:100A9000046F020E056F000E066F000E076F5EC139
:100AA00000F15FC101F160C102F161C103F1A0EC8D
:100AB0001DF003BF04D018BE02D018A0108C11A0E6
:100AC00067EF05F010BA67EF05F00F80108A0CC1D0
:100AD00000F10DC101F10EC102F10FC103F110C10E
:100AE00004F111C105F112C106F113C107F114C1DE
:100AF00008F115C109F116C10AF117C10BF135C191
:100B000034F112EF09F00392ABB2AB98AB8803015A
:100B100003EE00F080517F0BE92604C0EFFF802B2D
:100B20008151805D700BD8A48B8200008051815D63
:100B3000700BD8A48B9281518019D8B4079012EF12
:100B400009F0F2940101453F12EF09F0462B12EF34
:100B500009F09E900101533F12EF09F0542B12EF60
:100B600009F09E9211B820EF07F08BB4BFEF05F0AB
:100B700010ACBFEF05F08B84109CC0EF05F08B9498
:100B8000C3CF55F1C4CF56F1C28207B42AEF06F0A5
:100B900047C14BF148C14CF149C14DF14AC14EF139
:100BA0005EC162F15FC163F160C164F161C165F171
:100BB00096C1B6F197C1B7F198C1B8F199C1B9F131
:100BC0009AC1BAF19BC1BBF19CC1BCF19DC1BDF101
:100BD0009EC1BEF19FC1BFF1A0C1C0F1A1C1C1F1D1
:100BE000A2C1C2F1A3C1C3F1A4C1C4F1A5C1C5F1A1
:100BF000A6C1C6F1A7C1C7F1A8C1C8F1A9C1C9F171
:100C0000AAC1CAF1ABC1CBF1ACC1CCF1ADC1CDF140
:100C1000AEC1CEF1AFC1CFF1B0C1D0F1B1C1D1F110
:100C2000B2C1D2F1B3C1D3F1B4C1D4F1B5C1D5F1E0
:100C3000010155515B2756515C23E86A5D230E2E56
:100C40002AEF06F05CC157F15DC158F15B6B5C6B3C
:100C50005D6B078E0201002F12EF09F03C0E006F52
:100C60001950E00BE00AE866128817BE02D017B4EC
:100C7000108E00C10CF101C10DF102C10EF103C1D2
:100C80000FF104C110F105C111F106C112F107C144
:100C900013F108C114F109C115F10AC116F10BC114
:100CA00017F134C135F101018A675EEF06F08B67F9
:100CB0005EEF06F08C675EEF06F08D6762EF06F080
:100CC00092EF06F08EC100F18FC101F190C102F1E7
:100CD00091C103F10101010E046F000E056F000EBA
:100CE000066F000E076FA0EC1DF000C18EF101C170
:100CF0008FF102C190F103C191F1006787EF06F017
:100D0000016787EF06F0026787EF06F0036792EF4F
:100D100006F08AC18EF18BC18FF18CC190F18DC12B
:100D200091F10F80D57ED5BE6DD0D6CF47F1D7CF0C
:100D300048F145C149F1E86AE8CF4AF118BE02D04E
:100D400018A0108C109047C100F148C101F149C1B1
:100D500002F14AC103F101010A0E046F000E056F92
:100D6000000E066F000E076FA0EC1DF003AF1080A1
:100D7000010154A7C8EF06F00F9A0F9C0F9E0101C6
:100D8000000E5E6F600E5F6F3D0E606F080E616F4C
:100D9000010147BFD8EF06F04867D8EF06F0496772
:100DA000D8EF06F04A67D8EF06F0F288FDEF06F0BC
:100DB000F2985E6B5F6B606B616B966B976B986B79
:100DC000996B9A6B9B6B9C6B9D6B9E6B9F6BA06BE7
:100DD000A16BA26BA36BA46BA56BA66BA76BA86B97
:100DE000A96BAA6BAB6BAC6BAD6BAE6BAF6BB06B47
:100DF000B16BB26BB36BB46BB56BD76AD66A0101DA
:100E0000456B466B0CC100F10DC101F10EC102F141
:100E10000FC103F110C104F111C105F112C106F1B6
:100E200013C107F114C108F115C109F116C10AF186
:100E300017C10BF135C134F112EF09F012EF09F0CF
:100E40000201002F79EF08F0D59ED6CF47F1D7CF1A
:100E500048F145C149F1E86AE8CF4AF1D76AD66A54
:100E60000101456B466BD58E1950E00BE00AE86630
:100E7000128817BE02D017B4108E16AE1B8C00C19C
:100E80000CF101C10DF102C10EF103C10FF104C15A
:100E900010F105C111F106C112F107C113F108C12A
:100EA00014F109C115F10AC116F10BC117F134C1D2
:100EB00035F10FA0109A11B869EF07F00101620E29
:100EC000046F010E056F000E066F000E076F72EFC4
:100ED00007F00101A70E046F020E056F000E066FEA
:100EE000000E076F47C100F148C101F149C102F18D
:100EF0004AC103F1A0EC1DF003BF85EF07F018BE57
:100F000002D018A0108C11B00F800CC100F10DC1DF
:100F100001F10EC102F10FC103F110C104F111C1C1
:100F200005F112C106F113C107F114C108F115C191
:100F300009F116C10AF117C10BF135C134F10201F3
:100F40003C0E006F00C10CF101C10DF102C10EF1A8
:100F500003C10FF104C110F105C111F106C112F175
:100F600007C113F108C114F109C115F10AC116F145
:100F70000BC117F134C135F101018A67C7EF07F0E2
:100F80008B67C7EF07F08C67C7EF07F08D67CBEF74
:100F900007F0FBEF07F08EC100F18FC101F190C1A6
:100FA00002F191C103F10101010E046F000E056F02
:100FB000000E066F000E076FA0EC1DF000C18EF151
:100FC00001C18FF102C190F103C191F10067F0EF0F
:100FD00007F00167F0EF07F00267F0EF07F0036733
:100FE000FBEF07F08AC18EF18BC18FF18CC190F1BC
:100FF0008DC191F10F80109047C100F148C101F1FE
:1010000049C102F14AC103F101010A0E046F000E49
:10101000056F000E066F000E076FA0EC1DF003AF0A
:101020001080010154A721EF08F00F9A0F9C0F9E2A
:101030000101000E5E6F600E5F6F3D0E606F080E67
:10104000616F47C100F148C101F149C102F14AC1D4
:1010500003F10101140E046F050E056F000E066FFB
:10106000000E076FA0EC1DF003AF3AEF08F0F28816
:101070005FEF08F0F2985E6B5F6B606B616B966B75
:10108000976B986B996B9A6B9B6B9C6B9D6B9E6B34
:101090009F6BA06BA16BA26BA36BA46BA56BA66BE4
:1010A000A76BA86BA96BAA6BAB6BAC6BAD6BAE6B94
:1010B000AF6BB06BB16BB26BB36BB46BB56B0CC198
:1010C00000F10DC101F10EC102F10FC103F110C118
:1010D00004F111C105F112C106F113C107F114C1E8
:1010E00008F115C109F116C10AF117C10BF135C19B
:1010F00034F1BCEC21F01C661ED01BAE11D01B9E3F
:101100001C8E17AE07D0136A040E146E156A09EC14
:101110001FF011D0136A146A156A09EC1FF00BD086
:101120001BAC09D01B9C1C8C010E136E146A156A33
:10113000FDEC20F000D08BB4A5EF08F010ACA5EFCB
:1011400008F08B84109CA6EF08F08B94C3CF55F168
:10115000C4CF56F1C28207B410EF09F047C14BF17A
:1011600048C14CF149C14DF14AC14EF15EC162F135
:101170005FC163F160C164F161C165F196C1B6F10F
:1011800097C1B7F198C1B8F199C1B9F19AC1BAF153
:101190009BC1BBF19CC1BCF19DC1BDF19EC1BEF123
:1011A0009FC1BFF1A0C1C0F1A1C1C1F1A2C1C2F1F3
:1011B000A3C1C3F1A4C1C4F1A5C1C5F1A6C1C6F1C3
:1011C000A7C1C7F1A8C1C8F1A9C1C9F1AAC1CAF193
:1011D000ABC1CBF1ACC1CCF1ADC1CDF1AEC1CEF163
:1011E000AFC1CFF1B0C1D0F1B1C1D1F1B2C1D2F133
:1011F000B3C1D3F1B4C1D4F1B5C1D5F10101555199
:101200005B2756515C23E86A5D230E2E10EF09F030
:101210005CC157F15DC158F15B6B5C6B5D6B078E18
:1012200012EF09F002C0E0FF005001C0D8FF10002B
:10123000A6B218EF09F00CC0A9FF0BC0A8FFA69E2C
:10124000A69CA684F29E550EA76EAA0EA76EA68235
:10125000F28EA694A6B22AEF09F00C2A1200A96E0B
:10126000A69EA69CA680A8500C2A120004012C0E53
:10127000826F2FEC0BF09BEC1EF00C502FEC09F062
:10128000E8CF00F10C502FEC09F0E8CF01F101AFED
:101290004FEF09F00101FF0E026FFF0E036F3EECEE
:1012A0001EF029675BEF09F00401200E826F2FEC1E
:1012B0000BF060EF09F004012D0E826F2FEC0BF0A4
:1012C00068EC1CF01200076A0F6A106A116A126A51
:1012D0000F010E0EC16E860EC06E030EC26E0F01A0
:1012E000896A110E926E080E8A6EF10E936E8B6AE9
:1012F000980E946EF18EFC0E2FEC09F0E8CF0BF0F7
:101300000BA011800BA211820BA411840BA81188D1
:10131000C90E2FEC09F0E8CF16F0CA0E2FEC09F039
:10132000E8CF17F0CB0E2FEC09F0E8CF18F0CC0E79
:101330002FEC09F0E8CF19F01B6A1C6A0E6A010154
:101340005B6B5C6B5D6B576B586BF29A0101476B83
:10135000486B496B4A6B4B6B4C6B4D6B4E6B4F6BD9
:10136000506B516B526B456B466BD76AD66A0F0157
:10137000280ED56EF28A9D90B00ECD6E01015E6B87
:101380005F6B606B616B626B636B646B656B666BF1
:10139000676B686B696B536B546BCF6ACE6A0F9A3D
:1013A0000F9C0F9E9D80760ECA6E9D8202013C0EA0
:1013B000006FCC6A160E2FEC09F0E8CF00F1170E83
:1013C0002FEC09F0E8CF01F1180E2FEC09F0E8CF6F
:1013D00002F1190E2FEC09F0E8CF03F1010103AF80
:1013E0000CEF0AF09BEC1EF0160E0C6E00C10BF019
:1013F00018EC09F0170E0C6E01C10BF018EC09F097
:10140000180E0C6E02C10BF018EC09F0190E0C6EE0
:1014100003C10BF018EC09F000C18AF101C18BF196
:1014200002C18CF103C18DF100C18EF101C18FF1B8
:1014300002C190F103C191F11A0E2FEC09F0E8CF2F
:1014400000F11B0E2FEC09F0E8CF01F11C0E2FEC80
:1014500009F0E8CF02F11D0E2FEC09F0E8CF03F1FF
:10146000010103AF62EF0AF09BEC1EF01A0E0C6E46
:1014700000C10BF018EC09F01B0E0C6E01C10BF053
:1014800018EC09F01C0E0C6E02C10BF018EC09F000
:101490001D0E0C6E03C10BF018EC09F01A0E2FECA8
:1014A00009F0E8CF00F11B0E2FEC09F0E8CF01F1B5
:1014B0001C0E2FEC09F0E8CF02F11D0E2FEC09F005
:1014C000E8CF03F100C192F101C193F102C194F19F
:1014D00003C195F1240EAC6E900EAB6E240EAC6E73
:1014E000080EB86E000EB06E1F0EAF6E0401806B5A
:1014F000816B0F01900EAB6E0F019D8A0301806B13
:10150000816BC26B8B92136A146A156A9D86079071
:101510000001F28EF28C07B015EF1BF00FB0B1EFA7
:1015200014F010BEB1EF14F012B8B1EF14F00301D3
:10153000805181197F0BD8B415EF1BF013EE00F02A
:1015400081517F0BE126812BE7CFE8FFE00BD8B478
:1015500015EF1BF023EE82F0C2513F0BD926E7CFE7
:10156000DFFFC22BDF50780AD8A415EF1BF00780ED
:101570008EC100F18FC101F190C102F191C103F15F
:101580000101040E046F000E056F000E066F000EC1
:10159000076FA0EC1DF000AFD7EF0AF00101030EBA
:1015A0008E6F000E8F6F000E906F000E916F030113
:1015B0008251720AD8B498EF14F08251520AD8B40A
:1015C00098EF14F08251750AD8B498EF14F0825154
:1015D000630AD8B4CFEF17F08251690AD8B444EF48
:1015E00011F082517A0AD8B457EF12F08251490AA9
:1015F000D8B4E3EF10F08251500AD8B4F5EF0FF0F1
:101600008251700AD8B43BEF10F08251540AD8B41A
:1016100069EF10F08251740AD8B4B2EF10F0825121
:10162000410AD8B443EF0BF082516D0AD8B44DEFA4
:101630000FF082514D0AD8B466EF0FF08251730A51
:10164000D8B4C8EF13F08251530AD8B42DEF14F078
:101650008251590AD8B49EEF0EF006EF18F004013B
:1016600014EE00F080517F0BE12682C4E7FF802B4F
:10167000120004010D0E826F2FEC0BF00A0E826F28
:101680002FEC0BF012000401410E826F2FEC0BF0D7
:1016900003018351310AD8B4BEEF0DF00301835129
:1016A000320AD8B4EEEF0CF003018351330AD8B4F8
:1016B00077EF0CF003018351340AD8B467EF0BF0D5
:1016C00004013F0E826F2FEC0BF004EF18F0CC0EEC
:1016D0002FEC09F0E8CF0BF004012C0E826F2FECF9
:1016E0000BF003018451310AD8B48BEF0BF00301E6
:1016F0008451300AD8B48DEF0BF0030184514D0AA8
:10170000D8B497EF0BF003018451540AD8B49EEF7C
:101710000BF0B5EF0BF08A8401D08A940BAE04D0A5
:101720000BAC02D00BBA21D0E00E0B1218D01F0E5A
:101730000B168539E844E00B0B1211D0E00E0B16A6
:10174000DCEC1EF085C332F186C333F10101296B55
:10175000E9EC1EF060EC1EF000511F0B0B12CC0EDA
:101760000C6E0BC00BF018EC09F00401340E826F04
:101770002FEC0BF004012C0E826F2FEC0BF0CC0E33
:101780002FEC09F0E8CF19F08AB406D00401300E2E
:10179000826F2FEC0BF005D00401310E826F2FEC1D
:1017A0000BF004012C0E826F2FEC0BF01938E8407F
:1017B000070BE8CF82F40401300E82272FEC0BF0E8
:1017C00004012C0E826F2FEC0BF09BEC1EF01950D5
:1017D0001F0BE8CF00F13EEC1EF032C182F4040191
:1017E000300E82272FEC0BF033C182F40401300E4F
:1017F00082272FEC0BF004012C0E826F2FEC0BF0E4
:101800009BEC1EF02CC000F100AF0BD0FF0E016F5F
:10181000FF0E026FFF0E036F04012D0E826F2FEC7F
:101820000BF03EEC1EF031C182F40401300E822731
:101830002FEC0BF032C182F40401300E82272FEC22
:101840000BF033C182F40401300E82272FEC0BF031
:1018500004012C0E826F2FEC0BF09BEC1EF02BC0C2
:1018600000F13EEC1EF031C182F40401300E8227FB
:101870002FEC0BF032C182F40401300E82272FECE2
:101880000BF033C182F40401300E82272FEC0BF0F1
:1018900004012C0E826F2FEC0BF09BEC1EF02DC080
:1018A00000F100AF0BD0FF0E016FFF0E026FFF0EB5
:1018B000036F04012D0E826F2FEC0BF03EEC1EF037
:1018C00031C182F40401300E82272FEC0BF032C1BB
:1018D00082F40401300E82272FEC0BF033C182F426
:1018E0000401300E82272FEC0BF004EF18F0CB0E22
:1018F0002FEC09F0E8CF0BF004012C0E826F2FECD7
:101900000BF003018451450AD8B49BEF0CF003019E
:101910008451440AD8B49EEF0CF003018451300A7C
:10192000D8B4A1EF0CF003018451310AD8B4A5EF6B
:101930000CF0B0EF0CF00B9EAAEF0CF00B8EAAEFA0
:101940000CF0FC0E0B16AAEF0CF0FC0E0B160B8025
:10195000AAEF0CF0CB0E0C6E0BC00BF018EC09F0DC
:101960000401330E826F2FEC0BF004012C0E826FFA
:101970002FEC0BF0CB0E2FEC09F0E8CF18F018BECF
:10198000C9EF0CF00401450E826F2FEC0BF0CEEF87
:101990000CF00401440E826F2FEC0BF004012C0EAE
:1019A000826F2FEC0BF00401300E826F2FEC0BF0E6
:1019B00004012C0E826F2FEC0BF018B0E7EF0CF047
:1019C0000401300E826F2FEC0BF0ECEF0CF00401F1
:1019D000310E826F2FEC0BF004EF18F0CA0E2FECD3
:1019E00009F0E8CF0BF004012C0E826F2FEC0BF006
:1019F00003018451450AD8B42AEF0DF00301845144
:101A0000440AD8B42DEF0DF0030184514D0AD8B427
:101A100036EF0DF003018451410AD8B430EF0DF0D8
:101A200003018451460AD8B433EF0DF00301845109
:101A3000560AD8B43EEF0DF003018451500AD8B4D1
:101A400049EF0DF003018451520AD8B44CEF0DF068
:101A500055EF0DF00B9E4FEF0DF00B8E4FEF0DF08D
:101A60000B9C4FEF0DF00B8C4FEF0DF0FC0E0B1697
:101A700085C3E8FF030B0B124FEF0DF0C70E0B16DB
:101A800085C3E8FF070BE846E846E8460B124FEF30
:101A90000DF00B844FEF0DF00B944FEF0DF0CA0ECD
:101AA0000C6E0BC00BF018EC09F0CA0E2FEC09F00D
:101AB000E8CF17F00401320E826F2FEC0BF0040117
:101AC0002C0E826F2FEC0BF017BE6EEF0DF00401A1
:101AD000450E826F2FEC0BF073EF0DF00401440EF6
:101AE000826F2FEC0BF004012C0E826F2FEC0BF0A9
:101AF00017C0E8FF030BE8CF82F40401300E822701
:101B00002FEC0BF004012C0E826F2FEC0BF017BCA6
:101B100091EF0DF00401410E826F2FEC0BF096EF68
:101B20000DF00401460E826F2FEC0BF004012C0E19
:101B3000826F2FEC0BF017C0E8FF380BE842E84249
:101B4000E842E8CF82F40401300E82272FEC0BF03C
:101B500004012C0E826F2FEC0BF017B4B7EF0DF0D1
:101B60000401520E826F2FEC0BF0BCEF0DF004015C
:101B7000500E826F2FEC0BF004EF18F0C90E2FEC13
:101B800009F0E8CF0BF004012C0E826F2FEC0BF064
:101B900003018451450AD8B4DCEF0DF003018451F0
:101BA000440AD8B4DFEF0DF0030184514D0AD8B4D4
:101BB000E2EF0DF0F0EF0DF00B9EEAEF0DF00B8E63
:101BC000EAEF0DF0F80E0B1685C3E8FF070B0B12BA
:101BD000EAEF0DF0C90E0C6E0BC00BF018EC09F01B
:101BE0000401310E826F2FEC0BF004012C0E826F7A
:101BF0002FEC0BF0C90E2FEC09F0E8CF16F016BE53
:101C000006D00401450E826F2FEC0BF005D00401C5
:101C1000440E826F2FEC0BF004012C0E826F2FEC20
:101C20000BF016C0E8FF070BE8CF82F40401300E7A
:101C300082272FEC0BF004012C0E826F2FEC0BF09F
:101C400007809BEC1EF027C0E8FF003B00430043E9
:101C5000030B3EEC1EF033C182F40401300E8227E8
:101C60002FEC0BF004012C0E826F2FEC0BF09BEC91
:101C70001EF027C001F1019F019D28C000F1010164
:101C80003EEC1EF02FC182F40401300E82272FECAF
:101C90000BF030C182F40401300E82272FEC0BF0E0
:101CA00031C182F40401300E82272FEC0BF032C1D7
:101CB00082F40401300E82272FEC0BF033C182F442
:101CC0000401300E82272FEC0BF004012C0E826FE2
:101CD0002FEC0BF09BEC1EF029C001F12AC000F1A3
:101CE000D89001330033D8900133003301013EEC2A
:101CF0001EF02FC182F40401300E82272FEC0BF06E
:101D000030C182F40401300E82272FEC0BF031C178
:101D100082F40401300E82272FEC0BF032C182F4E2
:101D20000401300E82272FEC0BF033C182F4040142
:101D3000300E82272FEC0BF004EF18F0FC0E2FEC86
:101D400009F0E8CF0BF003018351520AD8B4D5EF64
:101D50000EF003018351720AD8B4D8EF0EF00301DC
:101D60008351500AD8B4DBEF0EF003018351700A9F
:101D7000D8B4DEEF0EF003018351550AD8B4E1EF79
:101D80000EF003018351750AD8B4E4EF0EF003019D
:101D90008351430AD8B4EDEF0EF003018351630A77
:101DA000D8B4F0EF0EF0F9EF0EF00B90F3EF0EF069
:101DB0000B80F3EF0EF00B92F3EF0EF00B82F3EFCC
:101DC0000EF00B94F3EF0EF00B84F3EF0EF00B9686
:101DD000F3EF0EF00B86F3EF0EF00B98F3EF0EF02F
:101DE0000B88F3EF0EF0FC0E0C6E0BC00BF018EC32
:101DF00009F00401590E826F2FEC0BF01190119233
:101E000011941198FC0E2FEC09F0E8CF0BF00BA009
:101E100011800BA211820BA411840BA8118811A0B0
:101E200019EF0FF00401520E826F2FEC0BF01EEF32
:101E30000FF00401720E826F2FEC0BF011A828EF47
:101E40000FF00401430E826F2FEC0BF02DEF0FF01B
:101E50000401630E826F2FEC0BF011A237EF0FF02D
:101E60000401500E826F2FEC0BF03CEF0FF00401D9
:101E7000700E826F2FEC0BF011A446EF0FF00401EF
:101E8000550E826F2FEC0BF04BEF0FF00401750E27
:101E9000826F2FEC0BF004EF18F004016D0E826FCF
:101EA0002FEC0BF003018351300AD8B4A5EF0FF0EB
:101EB00003018351310AD8B4B8EF0FF00301835105
:101EC000320AD8B4CBEF0FF006EF18F004014D0E34
:101ED000826F2FEC0BF0DCEC1EF084C331F185C374
:101EE00032F186C333F10101296BE9EC1EF060EC9D
:101EF0001EF003018351300AD8B48DEF0FF00301B7
:101F00008351310AD8B495EF0FF003018351320A9F
:101F1000D8B49DEF0FF006EF18F0FD0E0C6E00C167
:101F20000BF018EC09F0A5EF0FF0FE0E0C6E00C1DF
:101F30000BF018EC09F0B8EF0FF0FF0E0C6E00C1BB
:101F40000BF018EC09F0CBEF0FF00401300E826FAC
:101F50002FEC0BF004012C0E826F2FEC0BF09BEC9E
:101F60001EF0FD0E2FEC09F0E8CF00F1DCEF0FF0D2
:101F70000401310E826F2FEC0BF004012C0E826FE6
:101F80002FEC0BF09BEC1EF0FE0E2FEC09F0E8CFCF
:101F900000F1DCEF0FF00401320E826F2FEC0BF03A
:101FA0009BEC1EF004012C0E826F2FEC0BF0FF0E49
:101FB0002FEC09F0E8CF00F13EEC1EF031C182F4C5
:101FC0000401300E82272FEC0BF032C182F40401A1
:101FD000300E82272FEC0BF033C182F40401300E57
:101FE00082272FEC0BF004EF18F081A8E3EF10F03C
:101FF00083C32AF184C32BF185C32CF186C32DF151
:1020000087C32EF188C32FF189C330F18AC331F120
:102010008BC332F18CC333F10101E9EC1EF060ECAB
:102020001EF0160E0C6E00C10BF018EC09F0170E26
:102030000C6E01C10BF018EC09F0180E0C6E02C109
:102040000BF018EC09F0190E0C6E03C10BF018EC34
:1020500009F000C18AF101C18BF102C18CF103C109
:102060008DF100C18EF101C18FF102C190F103C168
:1020700091F1E3EF10F081A8E3EF10F083C32AF1B0
:1020800084C32BF185C32CF186C32DF187C32EF1B8
:1020900088C32FF189C330F18AC331F18BC332F188
:1020A0008CC333F10101E9EC1EF060EC1EF000C1BD
:1020B0008AF101C18BF102C18CF103C18DF100C124
:1020C0008EF101C18FF102C190F103C191F1E3EFF3
:1020D00010F081A8E3EF10F083C32AF184C32BF141
:1020E00085C32CF186C32DF187C32EF188C32FF150
:1020F00089C330F18AC331F18CC332F18DC333F11E
:102100000101E9EC1EF060EC1EF00101000E046F0D
:10211000000E056F010E066F000E076FB1EC1DF08B
:102120001A0E0C6E00C10BF018EC09F01B0E0C6EB1
:1021300001C10BF018EC09F01C0E0C6E02C10BF083
:1021400018EC09F01D0E0C6E03C10BF018EC09F031
:1021500000C192F101C193F102C194F103C195F163
:10216000E3EF10F081A8E3EF10F083C32AF184C3FA
:102170002BF185C32CF186C32DF187C32EF188C3C3
:102180002FF189C330F18AC331F18CC332F18DC391
:1021900033F10101E9EC1EF060EC1EF00101000ECC
:1021A000046F000E056F010E066F000E076FB1EC95
:1021B0001DF000C192F101C193F102C194F103C17C
:1021C00095F1E3EF10F0160E2FEC09F0E8CF00F1D7
:1021D000170E2FEC09F0E8CF01F1180E2FEC09F0E3
:1021E000E8CF02F1190E2FEC09F0E8CF03F13EEC35
:1021F0001EF021EC1CF00401730E826F2FEC0BF02B
:1022000004012C0E826F2FEC0BF08AC100F18BC100
:1022100001F18CC102F18DC103F13EEC1EF021EC05
:102220001CF00401730E826F2FEC0BF004012C0ED6
:10223000826F2FEC0BF01A0E2FEC09F0E8CF00F1B3
:102240001B0E2FEC09F0E8CF01F11C0E2FEC09F06A
:10225000E8CF02F11D0E2FEC09F0E8CF03F121ECDD
:1022600018F004012C0E826F2FEC0BF092C100F1DC
:1022700093C101F194C102F195C103F121EC18F071
:1022800039EC0BF006EF18F00401690E826F2FECA9
:102290000BF004012C0E826F2FEC0BF00101040EE9
:1022A000006F000E016F000E026F000E036F3EEC18
:1022B0001EF02CC182F40401300E82272FEC0BF0AB
:1022C0002DC182F40401300E82272FEC0BF02EC1B9
:1022D00082F40401300E82272FEC0BF02FC182F420
:1022E0000401300E82272FEC0BF030C182F4040180
:1022F000300E82272FEC0BF031C182F40401300E36
:1023000082272FEC0BF032C182F40401300E8227B9
:102310002FEC0BF033C182F40401300E82272FEC36
:102320000BF004012C0E826F2FEC0BF00101030E59
:10233000006F000E016F000E026F000E036F3EEC87
:102340001EF02CC182F40401300E82272FEC0BF01A
:102350002DC182F40401300E82272FEC0BF02EC128
:1023600082F40401300E82272FEC0BF02FC182F48F
:102370000401300E82272FEC0BF030C182F40401EF
:10238000300E82272FEC0BF031C182F40401300EA5
:1023900082272FEC0BF032C182F40401300E822729
:1023A0002FEC0BF033C182F40401300E82272FECA6
:1023B0000BF004012C0E826F2FEC0BF001012C0EA0
:1023C000006F000E016F000E026F000E036F3EECF7
:1023D0001EF02CC182F40401300E82272FEC0BF08A
:1023E0002DC182F40401300E82272FEC0BF02EC198
:1023F00082F40401300E82272FEC0BF02FC182F4FF
:102400000401300E82272FEC0BF030C182F404015E
:10241000300E82272FEC0BF031C182F40401300E14
:1024200082272FEC0BF032C182F40401300E822798
:102430002FEC0BF033C182F40401300E82272FEC15
:102440000BF004012C0E826F2FEC0BF0200EF86EB7
:10245000F76AF66A04010900F5CF82F42FEC0BF05D
:102460000900F5CF82F42FEC0BF00900F5CF82F4D0
:102470002FEC0BF00900F5CF82F42FEC0BF00900E4
:10248000F5CF82F42FEC0BF00900F5CF82F42FEC9E
:102490000BF00900F5CF82F42FEC0BF00900F5CF1B
:1024A00082F42FEC0BF039EC0BF006EF18F08351AF
:1024B000630AD8A406EF18F08451610AD8A406EF85
:1024C00018F085516C0AD8A406EF18F08651410A1D
:1024D00042E08651440A1BE08651420AD8B4BEEF5E
:1024E00012F08651350AD8B490EF19F08651360AA9
:1024F000D8B4E5EF19F08651370AD8B44EEF1AF088
:102500008651380AD8B4ACEF1AF006EF18F00798E5
:10251000079A04017A0E826F2FEC0BF00401780EFB
:10252000826F2FEC0BF00401640E826F2FEC0BF026
:1025300081A8A2EF12F00401550E826F2FEC0BF070
:10254000A7EF12F004014C0E826F2FEC0BF039EC68
:102550000BF006EF18F00788079A04017A0E826FD5
:102560002FEC0BF00401410E826F2FEC0BF00401F5
:10257000610E826F2FEC0BF098EF12F00798078A2C
:1025800004017A0E826F2FEC0BF00401420E826F71
:102590002FEC0BF00401610E826F2FEC0BF098EF23
:1025A00012F001016667DCEF12F06767DCEF12F0F2
:1025B0006867DCEF12F0696715D04F67E7EF12F03C
:1025C0005067E7EF12F05167E7EF12F052670AD059
:1025D0000101000E006F000E016F000E026F000E71
:1025E000036F120011B80AD00101620E046F010ED0
:1025F000056F000E066F000E076F09D00101A70ED0
:10260000046F020E056F000E066F000E076F66C1A5
:1026100000F167C101F168C102F169C103F1A0ECE9
:102620001DF003BF84EF13F0119A119C0101000EFD
:10263000046FA80E056F550E066F020E076F66C178
:1026400000F167C101F168C102F169C103F166C11E
:1026500086F167C187F168C188F169C189F1A0EC91
:102660001DF003BF0BD00101000E866FA80E876F0F
:10267000550E886F020E896F118A119C0E0E2FEC79
:1026800009F0E8CF18F10F0E2FEC09F0E8CF19F19F
:10269000100E2FEC09F0E8CF1AF1110E2FEC09F013
:1026A000E8CF1BF1E9EC1CF086C104F187C105F10C
:1026B00088C106F189C107F1A0EC1DF00782ADECDD
:1026C0001CF0E9EC1CF00792ADEC1CF086C100F1A7
:1026D00087C101F188C102F189C103F10792ADEC14
:1026E0001CF0CC0E046FE00E056F870E066F050E12
:1026F000076FA0EC1DF000C118F101C119F102C172
:102700001AF103C11BF13BD0119C119A0101800EFB
:10271000006F1A0E016F060E026F000E036F4FC19D
:1027200004F150C105F151C106F152C107F1A0EC0D
:102730001DF003AF05D09BEC1EF0118C119A120016
:102740000E0E2FEC09F0E8CF18F10F0E2FEC09F068
:10275000E8CF19F1100E2FEC09F0E8CF1AF1110EA5
:102760002FEC09F0E8CF1BF14FC100F150C101F18E
:1027700051C102F152C103F10782ADEC1CF018C146
:1027800000F119C101F11AC102F11BC103F11200DC
:102790000401730E826F2FEC0BF004012C0E826F7C
:1027A0002FEC0BF0078462C166F163C167F164C16D
:1027B00068F165C169F14BC14FF14CC150F14DC198
:1027C00051F14EC152F157C159F158C15AF1079414
:1027D000EEEC13F039EC0BF006EF18F066C100F1E7
:1027E00067C101F168C102F169C103F101013EEC69
:1027F0001EF021EC1CF00401630E826F2FEC0BF035
:1028000004012C0E826F2FEC0BF04FC100F150C170
:1028100001F151C102F152C103F101013EEC1EF080
:1028200021EC1CF00401660E826F2FEC0BF004010A
:102830002C0E826F2FEC0BF09BEC1EF059C100F1B7
:102840005AC101F101013EEC1EF021EC1CF0040123
:10285000740E826F2FEC0BF0120010820401530EE5
:10286000826F2FEC0BF004012C0E826F2FEC0BF01B
:1028700083C32AF184C32BF185C32CF186C32DF1C8
:1028800087C32EF188C32FF189C330F18AC331F198
:102890008BC332F18CC333F10101E9EC1EF060EC23
:1028A0001EF000C166F101C167F102C168F103C108
:1028B00069F18EC32AF18FC32BF190C32CF191C320
:1028C0002DF192C32EF193C32FF194C330F195C330
:1028D00031F196C332F197C333F10101E9EC1EF0F7
:1028E00060EC1EF000C14FF101C150F102C151F185
:1028F00003C152F1DCEC1EF099C32FF19AC330F101
:102900009BC331F19CC332F19DC333F10101E9EC6A
:102910001EF060EC1EF000C159F101C15AF1EEEC5D
:1029200013F004012C0E826F2FEC0BF0A5EF14F0C6
:10293000118E18B0108C17BE02D017A4108E8251C1
:10294000520A02E10F8201D00F928251750A02E110
:10295000108401D010948251550A02E1108601D0F2
:10296000109611A003D011A401D01084078410B2D6
:1029700013EF15F010A4FFEF14F0B6C166F1B7C164
:1029800067F1B8C168F1B9C169F1BAC16AF1BBC1F7
:102990006BF1BCC16CF1BDC16DF1BEC16EF1BFC1C7
:1029A0006FF1C0C170F1C1C171F1C2C172F1C3C197
:1029B00073F1C4C174F1C5C175F1C6C176F1C7C167
:1029C00077F1C8C178F1C9C179F1CAC17AF1CBC137
:1029D0007BF1CCC17CF1CDC17DF1CEC17EF1CFC107
:1029E0007FF1D0C180F1D1C181F1D2C182F1D3C1D7
:1029F00083F1D4C184F1D5C185F107EF15F062C12F
:102A000066F163C167F164C168F165C169F14BC1E9
:102A10004FF14CC150F14DC151F14EC152F157C16E
:102A200059F158C15AF107940FA035EF15F0010183
:102A3000926722EF15F0936722EF15F0946722EF6B
:102A400015F0956726EF15F035EF15F0D1EC12F083
:102A500092C104F193C105F194C106F195C107F14A
:102A6000A0EC1DF003BFCCEF17F0D1EC12F0010188
:102A7000000E046F000E056F010E066F000E076F4B
:102A8000D1EC1DF011A02CD011A22AD03EEC1EF0EA
:102A9000296701D007D004012D0E826F2FEC0BF0B7
:102AA000CAEF17F030C182F40401300E82272FECF8
:102AB0000BF031C182F40401300E82272FEC0BF0B1
:102AC00032C182F40401300E82272FEC0BF033C1A7
:102AD00082F40401300E82272FEC0BF0CAEF17F0BE
:102AE00012A8C5D0129819C01AF01A3A1A42070E45
:102AF0001A1600011A50000AD8B403EF16F00001AC
:102B00001A50010AD8B48FEF15F000011A50020ACA
:102B1000D8B48DEF15F035EF16F035EF16F09BECCD
:102B20001EF029C001F12AC000F1D8900133003312
:102B3000D890013300330101630E046F000E056F5E
:102B4000000E066F000E076FD1EC1DF0280E046F0B
:102B5000000E056F000E066F000E076FA0EC1DF053
:102B600000C12CF09BEC1EF027C001F1019F019DDC
:102B700028C000F10101A40E046F000E056F000EC5
:102B8000066F000E076FD1EC1DF000C12BF000C1E5
:102B900004F101C105F102C106F103C107F1640EA0
:102BA000006F000E016F000E026F000E036FA0ECAD
:102BB0001DF0050E046F000E056F000E066F000E6F
:102BC000076FD1EC1DF000C104F101C105F102C194
:102BD00006F103C107F19BEC1EF02CC000F1A0EC44
:102BE0001DF000C12DF02DC0E8FF050F2C5C03E7A0
:102BF0008A8435EF16F02DC0E8FF0A0F2C5C01E641
:102C00008A9435EF16F000C124F101C125F102C10B
:102C100026F103C127F19BEC1EF0A1EC1EF0195028
:102C20001F0BE8CF00F10101640E046F000E056F69
:102C3000000E066F000E076FB1EC1DF024C104F109
:102C400025C105F126C106F127C107F1A0EC1DF051
:102C500003BF02D08A9401D08A8424C100F125C127
:102C600001F126C102F127C103F1CCEF17F000C139
:102C700024F101C125F102C126F103C127F110AEF3
:102C80004CD0109E00C108F101C109F102C10AF146
:102C900003C10BF13EEC1EF030C1D6F131C1D7F1CA
:102CA00032C1D8F133C1D9F108C100F109C101F134
:102CB0000AC102F10BC103F101016C0E046F070E92
:102CC000056F000E066F000E076FA0EC1DF003BF2E
:102CD00004D00101550EDA6F1CD008C100F109C102
:102CE00001F10AC102F10BC103F10101A40E046F4D
:102CF000060E056F000E066F000E076FA0EC1DF0AC
:102D000003BF04D001017F0EDA6F03D00101FF0E73
:102D1000DA6F1B8E11AECCEF17F024C100F125C184
:102D200001F126C102F127C103F110A49FEF16F0B3
:102D30000401750E826F2FEC0BF0A4EF16F0040166
:102D4000720E826F2FEC0BF004012C0E826F2FECB1
:102D50000BF03EEC1EF02967B3EF16F00401200ED5
:102D6000826FB6EF16F004012D0E826F2FEC0BF080
:102D700030C182F40401300E82272FEC0BF031C1F8
:102D800082F40401300E82272FEC0BF004012E0E8A
:102D9000826F2FEC0BF032C182F40401300E8227D7
:102DA0002FEC0BF033C182F40401300E82272FEC9C
:102DB0000BF004016D0E826F2FEC0BF004012C0E52
:102DC000826F2FEC0BF04FC100F150C101F151C1E6
:102DD00002F152C103F101013EEC1EF021EC1CF0A6
:102DE0000401480E826F2FEC0BF004017A0E826F03
:102DF0002FEC0BF004012C0E826F2FEC0BF066C150
:102E000000F167C101F168C102F169C103F101017B
:102E10003EEC1EF021EC1CF00401630E826F2FECDF
:102E20000BF004012C0E826F2FEC0BF066C100F149
:102E300067C101F168C102F169C103F101010A0E24
:102E4000046F000E056F000E066F000E076FB1ECE9
:102E50001DF0000E046F120E056F000E066F000EBF
:102E6000076FD1EC1DF03EEC1EF02AC182F4040184
:102E7000300E82272FEC0BF02BC182F40401300EB0
:102E800082272FEC0BF02CC182F40401300E822734
:102E90002FEC0BF02DC182F40401300E82272FECB1
:102EA0000BF02EC182F40401300E82272FEC0BF0C0
:102EB0002FC182F40401300E82272FEC0BF030C1B9
:102EC00082F40401300E82272FEC0BF004012E0E49
:102ED000826F2FEC0BF031C182F40401300E822797
:102EE0002FEC0BF032C182F40401300E82272FEC5C
:102EF0000BF033C182F40401300E82272FEC0BF06B
:102F00000401730E826F2FEC0BF004012C0E826F04
:102F10002FEC0BF09BEC1EF059C100F15AC101F1EE
:102F200030EC19F00FB298EF17F00FA0CAEF17F0BE
:102F300004012C0E826F2FEC0BF0200EF86EF76A56
:102F4000F66A04010900F5CF82F42FEC0BF00900BA
:102F5000F5CF82F42FEC0BF00900F5CF82F42FECC3
:102F60000BF00900F5CF82F42FEC0BF00900F5CF40
:102F700082F42FEC0BF00900F5CF82F42FEC0BF06C
:102F80000900F5CF82F42FEC0BF00900F5CF82F4A5
:102F90002FEC0BF039EC0BF00F9006EF18F004015A
:102FA000630E826F2FEC0BF004012C0E826F2FEC5E
:102FB0000BF00CEC18F004012C0E826F2FEC0BF0D0
:102FC0007FEC18F004012C0E826F2FEC0BF0FBEC61
:102FD00018F004012C0E826F2FEC0BF00101F80E9B
:102FE000006FCD0E016F660E026F030E036F21ECB2
:102FF00018F004012C0E826F2FEC0BF011EC19F07D
:1030000039EC0BF006EF18F039EC0BF00301C26B52
:103010000790109215EF1BF0D8900E0E2FEC09F0D0
:10302000E8CF00F10F0E2FEC09F0E8CF01F1100E00
:103030002FEC09F0E8CF02F1110E2FEC09F0E8CFE8
:1030400003F10101000E046F000E056F010E066F03
:10305000000E076FD1EC1DF03EEC1EF02AC182F489
:103060000401300E82272FEC0BF02BC182F40401F7
:10307000300E82272FEC0BF02CC182F40401300EAD
:1030800082272FEC0BF02DC182F40401300E822731
:103090002FEC0BF02EC182F40401300E82272FECAE
:1030A0000BF02FC182F40401300E82272FEC0BF0BD
:1030B00030C182F40401300E82272FEC0BF031C1B5
:1030C00082F40401300E82272FEC0BF004012E0E47
:1030D000826F2FEC0BF032C182F40401300E822794
:1030E0002FEC0BF033C182F40401300E82272FEC59
:1030F0000BF004016D0E826F2FEC0BF01200120E1C
:103100002FEC09F0E8CF00F1130E2FEC09F0E8CF17
:1031100001F1140E2FEC09F0E8CF02F1150E2FEC9F
:1031200009F0E8CF03F101010A0E046F000E056FEC
:10313000000E066F000E076FB1EC1DF0000E046F5D
:10314000120E056F000E066F000E076FD1EC1DF01A
:103150003EEC1EF02AC182F40401300E82272FECCF
:103160000BF02BC182F40401300E82272FEC0BF000
:103170002CC182F40401300E82272FEC0BF02DC1FC
:1031800082F40401300E82272FEC0BF02EC182F462
:103190000401300E82272FEC0BF02FC182F40401C2
:1031A000300E82272FEC0BF030C182F40401300E78
:1031B00082272FEC0BF004012E0E826F2FEC0BF008
:1031C00031C182F40401300E82272FEC0BF032C1A2
:1031D00082F40401300E82272FEC0BF033C182F40D
:1031E0000401300E82272FEC0BF00401730E826F66
:1031F0002FEC0BF012000A0E2FEC09F0E8CF00F1D3
:103200000B0E2FEC09F0E8CF01F10C0E2FEC09F0BA
:10321000E8CF02F10D0E2FEC09F0E8CF03F130EF0B
:1032200019F0060E2FEC09F0E8CF00F1070E2FEC95
:1032300009F0E8CF01F1080E2FEC09F0E8CF02F118
:10324000090E2FEC09F0E8CF03F130EF19F001017E
:103250009BEC1EF0078457C100F158C101F107949F
:103260000101E80E046F800E056F000E066F000E60
:10327000076FB1EC1DF0000E046F040E056F000E19
:10328000066F000E076FD1EC1DF0880E046F130E51
:10329000056F000E066F000E076FA0EC1DF00A0E02
:1032A000046F000E056F000E066F000E076FD1EC65
:1032B0001DF03EEC1EF00101296764EF19F00401D6
:1032C000200E826F67EF19F004012D0E826F2FEC34
:1032D0000BF030C182F40401300E82272FEC0BF08A
:1032E00031C182F40401300E82272FEC0BF032C181
:1032F00082F40401300E82272FEC0BF004012E0E15
:10330000826F2FEC0BF033C182F40401300E822760
:103310002FEC0BF00401430E826F2FEC0BF0120028
:1033200087C32AF188C32BF189C32CF18AC32DF1FD
:103330008BC32EF18CC32FF18DC330F18EC331F1CD
:1033400090C332F191C333F10101296BE9EC1EF016
:1033500060EC1EF00101000E046F000E056F010EFF
:10336000066F000E076FB1EC1DF00E0E0C6E00C163
:103370000BF018EC09F00F0E0C6E01C10BF018ECFD
:1033800009F0100E0C6E02C10BF018EC09F0110ED2
:103390000C6E03C10BF018EC09F004017A0E826F79
:1033A0002FEC0BF004012C0E826F2FEC0BF00401BC
:1033B000350E826F2FEC0BF004012C0E826F2FEC78
:1033C0000BF00CEC18F0A7EF12F087C32AF188C3BA
:1033D0002BF189C32CF18AC32DF18BC32EF18CC341
:1033E0002FF18DC330F18EC331F190C332F191C30F
:1033F00033F10101296BE9EC1EF060EC1EF0880E40
:10340000046F130E056F000E066F000E076FA5EC1C
:103410001DF0000E046F040E056F000E066F000E07
:10342000076FB1EC1DF00101E80E046F800E056F0F
:10343000000E066F000E076FD1EC1DF00A0E0C6E29
:1034400000C10BF018EC09F00B0E0C6E01C10BF073
:1034500018EC09F00C0E0C6E02C10BF018EC09F020
:103460000D0E0C6E03C10BF018EC09F004017A0E7E
:10347000826F2FEC0BF004012C0E826F2FEC0BF0FF
:103480000401360E826F2FEC0BF004012C0E826FBC
:103490002FEC0BF0FBEC18F0A7EF12F087C32AF12A
:1034A00088C32BF189C32CF18AC32DF18BC32EF174
:1034B0008CC32FF18DC330F18FC331F190C332F142
:1034C00091C333F10101E9EC1EF060EC1EF0000E37
:1034D000046F120E056F000E066F000E076FB1EC41
:1034E0001DF001010A0E046F000E056F000E066F3D
:1034F000000E076FD1EC1DF0120E0C6E00C10BF028
:1035000018EC09F0130E0C6E01C10BF018EC09F069
:10351000140E0C6E02C10BF018EC09F0150E0C6EB7
:1035200003C10BF018EC09F004017A0E826F2FEC46
:103530000BF004012C0E826F2FEC0BF00401370E00
:10354000826F2FEC0BF004012C0E826F2FEC0BF02E
:103550007FEC18F0A7EF12F087C32AF188C32BF194
:1035600089C32CF18AC32DF18BC32EF18CC32FF1AB
:103570008DC330F18EC331F190C332F191C333F179
:103580000101296BE9EC1EF060EC1EF0880E046F5F
:10359000130E056F000E066F000E076FA5EC1DF0F1
:1035A000000E046F040E056F000E066F000E076F0D
:1035B000B1EC1DF00101E80E046F800E056F000EE6
:1035C000066F000E076FD1EC1DF0060E0C6E00C1E9
:1035D0000BF018EC09F0070E0C6E01C10BF018ECA3
:1035E00009F0080E0C6E02C10BF018EC09F0090E80
:1035F0000C6E03C10BF018EC09F004017A0E826F17
:103600002FEC0BF004012C0E826F2FEC0BF0040159
:10361000380E826F2FEC0BF004012C0E826F2FEC12
:103620000BF011EC19F0A7EF12F081A8D3EF1BF00B
:1036300007A88CEF1BF00101800E006F1A0E016FBE
:10364000060E026F000E036F4BC104F14CC105F171
:103650004DC106F14EC107F1A0EC1DF003BFD3EF41
:103660001BF01BEC1CF04BC100F14CC101F14DC132
:1036700002F14EC103F10782ADEC1CF018C104F158
:1036800019C105F11AC106F11BC107F1F80E006F4F
:10369000CD0E016F660E026F030E036FA0EC1DF0DE
:1036A0000E0E0C6E00C10BF018EC09F00F0E0C6E34
:1036B00001C10BF018EC09F0100E0C6E02C10BF0FA
:1036C00018EC09F0110E0C6E03C10BF018EC09F0A8
:1036D000078401019BEC1EF057C100F158C101F1B4
:1036E00007940A0E0C6E00C10BF018EC09F00B0EDB
:1036F0000C6E01C10BF018EC09F00C0E0C6E02C13F
:103700000BF018EC09F00D0E0C6E03C10BF018EC69
:1037100009F00798D3EF1BF007AAD3EF1BF007843B
:1037200001019BEC1EF057C100F158C101F1079453
:10373000060E0C6E00C10BF018EC09F0070E0C6EB3
:1037400001C10BF018EC09F0080E0C6E02C10BF071
:1037500018EC09F0090E0C6E03C10BF018EC09F01F
:10376000078462C100F163C101F164C102F165C166
:1037700003F10794120E0C6E00C10BF018EC09F067
:10378000130E0C6E01C10BF018EC09F0140E0C6E48
:1037900002C10BF018EC09F0150E0C6E03C10BF012
:1037A00018EC09F0079A0401805181197F0B0BE096
:1037B0009EA809D014EE00F081517F0BE126E7505E
:1037C000812B0F01AD6E8BEF0AF018C100F119C10A
:1037D00001F11AC102F11BC103F1000E046F000ECA
:1037E000056F010E066F000E076FD1EC1DF029A1C9
:1037F00010EF1CF02051D8B410EF1CF018C100F1EC
:1038000019C101F11AC102F11BC103F1000E046FCD
:10381000000E056F0A0E066F000E076FD1EC1DF04B
:103820001200010104510013055101130651021346
:103830000751031312000101186B196B1A6B1B6BF4
:1038400012002AC182F40401300E82272FEC0BF003
:103850002BC182F40401300E82272FEC0BF02CC117
:1038600082F40401300E82272FEC0BF02DC182F47C
:103870000401300E82272FEC0BF02EC182F40401DC
:10388000300E82272FEC0BF02FC182F40401300E92
:1038900082272FEC0BF030C182F40401300E822716
:1038A0002FEC0BF031C182F40401300E82272FEC93
:1038B0000BF032C182F40401300E82272FEC0BF0A2
:1038C00033C182F40401300E82272FEC0BF012007A
:1038D0002FC182F40401300E82272FEC0BF030C18F
:1038E00082F40401300E82272FEC0BF031C182F4F8
:1038F0000401300E82272FEC0BF032C182F4040158
:10390000300E82272FEC0BF033C182F40401300E0D
:1039100082272FEC0BF01200060E1D6E060E1E6E97
:10392000060E1F6E1D2E92EF1CF01E2E92EF1CF045
:103930001F2E92EF1CF08B84020E1D6E020E1E6E67
:10394000020E1F6E1D2EA2EF1CF01E2EA2EF1CF009
:103950001F2EA2EF1CF08B9412000101005305E111
:10396000015303E1025301E1002B70EC1DF09BECCD
:103970001EF03951006F3A51016F420E046F4B0E29
:10398000056F000E066F000E076FB1EC1DF000C151
:1039900004F101C105F102C106F103C107F118C12B
:1039A00000F119C101F11AC102F11BC103F107B203
:1039B000DEEF1CF0A5EC1DF0E0EF1CF0A0EC1DF01C
:1039C00000C118F101C119F102C11AF103C11BF1C3
:1039D00012009BEC1EF059C100F15AC101F1060E14
:1039E0002FEC09F0E8CF04F1070E2FEC09F0E8CF37
:1039F00005F1080E2FEC09F0E8CF06F1090E2FECC7
:103A000009F0E8CF07F1A0EC1DF000C124F101C1DD
:103A100025F102C126F103C127F1290E046F000E22
:103A2000056F000E066F000E076FB1EC1DF0EE0E75
:103A3000046F430E056F000E066F000E076FA5ECB6
:103A40001DF024C104F125C105F126C106F127C1ED
:103A500007F1B1EC1DF000C11CF101C11DF102C163
:103A60001EF103C11FF1120E2FEC09F0E8CF04F193
:103A7000130E2FEC09F0E8CF05F1140E2FEC09F02E
:103A8000E8CF06F1150E2FEC09F0E8CF07F10D0E87
:103A9000006F000E016F000E026F000E036FB1EC9D
:103AA0001DF0180E046F000E056F000E066F000E5D
:103AB000076FD1EC1DF01CC104F11DC105F11EC141
:103AC00006F11FC107F1A5EC1DF06A0E046F2A0E66
:103AD000056F000E066F000E076FA0EC1DF01200C0
:103AE000BF0EFA6E200E3A6F396BD890003701374F
:103AF00002370337D8B081EF1DF03A2F76EF1DF073
:103B000039073A070353D8B412000331070B800971
:103B10003F6F03390F0B010F396F80EC5FF0406F7F
:103B2000390580EC5FF0405D405F396B3F33D8B0C2
:103B3000392739333FA996EF1DF04051392712003C
:103B40000101C0EC1EF0D8B01200010103510719A9
:103B5000346F83EC1EF0D8900751031934AF800FF7
:103B600012000101346BA7EC1EF0D8A0BDEC1EF0D2
:103B7000D8B0120092EC1EF09BEC1EF01F0E366FB8
:103B8000D3EC1EF00B35D8B083EC1EF0D8A0033573
:103B9000D8B01200362FC0EF1DF034B1AAEC1EF0E1
:103BA00012000101346B04510511061107110008C0
:103BB000D8A0A7EC1EF0D8A0BDEC1EF0D8B0120023
:103BC000086B096B0A6B0B6BD3EC1EF01F0E366F84
:103BD000D3EC1EF007510B5DD8A4FBEF1DF006518E
:103BE0000A5DD8A4FBEF1DF00551095DD8A4FBEFD9
:103BF0001DF00451085DD8A00EEF1EF00451085FBF
:103C00000551D8A0053D095F0651D8A0063D0A5FC1
:103C10000751D8A0073D0B5FD8900081362FE8EF01
:103C20001DF034B1AAEC1EF0346BA7EC1EF0D89056
:103C3000D7EC1EF007510B5DD8A42BEF1EF00651F8
:103C40000A5DD8A42BEF1EF00551095DD8A42BEF17
:103C50001EF00451085DD8A03AEF1EF0003F3AEF85
:103C60001EF0013F3AEF1EF0023F3AEF1EF0032B29
:103C7000D8B4120034B1AAEC1EF012000101346B6A
:103C8000A7EC1EF0D8B01200DCEC1EF0200E366F50
:103C9000003701370237033711EE33F00A0E376F62
:103CA000E7360A0EE75CD8B0E76EE552372F50EFE3
:103CB0001EF0362F48EF1EF034B12981D890120043
:103CC00001010A0E346F200E366F11EE29F03451C7
:103CD000376F0A0ED890E652D8B0E726E732372F72
:103CE0006BEF1EF00333023301330033362F65EFE1
:103CF0001EF0E750FF0FD8A00335D8B0120029B14D
:103D0000AAEC1EF01200045100270551D8B0053D61
:103D100001270651D8B0063D02270751D8B0073D0C
:103D2000032712000051086F0151096F02510A6FF9
:103D300003510B6F12000101006B016B026B036BEF
:103D400012000101046B056B066B076B1200033553
:103D5000D8A012000351800B001F011F021F031F78
:103D6000003FBAEF1EF0013FBAEF1EF0023FBAEF7C
:103D70001EF0032B342B032512000735D8A01200A8
:103D80000751800B041F051F061F071F043FD0EFBC
:103D90001EF0053FD0EF1EF0063FD0EF1EF0072BC0
:103DA000342B072512000037013702370337083755
:103DB00009370A370B3712000101296B2A6B2B6B6D
:103DC0002C6B2D6B2E6B2F6B306B316B326B336B1F
:103DD000120001012A510F0B2A6F2B510F0B2B6F71
:103DE0002C510F0B2C6F2D510F0B2D6F2E510F0BD4
:103DF0002E6F2F510F0B2F6F30510F0B306F315132
:103E00000F0B316F32510F0B326F33510F0B336F7A
:103E1000120000011550FF0A01E11200390EC86EB0
:103E2000800EC76E280EC66E000EC56E1450000AB6
:103E3000D8B444EF1FF01450010AD8B45DEF1FF05E
:103E40001450020AD8B476EF1FF01450030AD8B405
:103E50008FEF1FF01450040AD8B4B7EF1FF01450BE
:103E6000050AD8B4D0EF1FF01450060AD8B4E9EF11
:103E70001FF01450070AD8B402EF20F01450080ABB
:103E8000D8B41BEF20F012001550000AD8B43AEF56
:103E900020F01550010AD8B43EEF20F01550020A68
:103EA000D8B442EF20F01550030AD8B446EF20F002
:103EB0001550040AD8B4B5EF20F01550000AD8B454
:103EC0004AEF20F01550010AD8B44EEF20F01550FB
:103ED000020AD8B452EF20F01550030AD8B456EFB6
:103EE00020F01550040AD8B4B5EF20F01550000AA0
:103EF000D8B45AEF20F01550010AD8B45EEF20F084
:103F00001550020AD8B462EF20F01550030AD8B455
:103F100066EF20F01550040AD8B4B5EF20F0155024
:103F2000000AD8B473EF20F01550010AD8B477EF27
:103F300020F01550020AD8B47BEF20F01550030A88
:103F4000D8B48FEF20F01550040AD8B493EF20F0C6
:103F50001550050AD8B497EF20F01550060AD8B4CA
:103F60009BEF20F01550070AD8B49EEF20F01550B3
:103F7000000AD8B4A2EF20F01550010AD8B4A6EF79
:103F800020F01550020AD8B4AAEF20F01550030A09
:103F9000D8B4AEEF20F01550040AD8B4B1EF20F039
:103FA0001550000AD8B4B9EF20F01550010AD8B462
:103FB000BDEF20F01550020AD8B4C1EF20F0155023
:103FC000030AD8B4C5EF20F01550040AD8B4B5EFF1
:103FD00020F01550000AD8B4CFEF20F01550010A98
:103FE000D8B4D3EF20F01550020AD8B4D7EF20F0A0
:103FF0001550030AD8B4DBEF20F01550040AD8B4EA
:10400000B5EF20F01550000AD8B4DCEF20F01550C1
:10401000010AD8B4E0EF20F01550020AD8B4E4EF5A
:1040200020F01550030AD8B4E8EF20F01550040A28
:10403000D8B4B5EF20F01550000AD8B4E9EF20F05D
:104040001550010AD8B4EDEF20F01550020AD8B48B
:10405000F1EF20F01550030AD8B4F5EF20F0155019
:10406000040AD8B4F6EF20F01550050AD8B4F9EFD9
:1040700020F012009E96C580152A1200E20EC96E2D
:10408000152A1200770EC96E152A1200020EC96E8B
:10409000152A12009E96C580152A1200E20EC96EDE
:1040A000152A1200790EC96E152A1200000EC96E6B
:1040B000152A12009E96C580152A1200E20EC96EBE
:1040C000152A12007A0EC96E152A120017BC03D0E9
:1040D000DAC1E8FF04D01750E844E8441F09E8CFEC
:1040E000C9FF152A12009E96C580152A1200E20EFD
:1040F000C96E152A120011BA03D011BC01D003D029
:10410000050E146E3ED00101D6678BEF20F0100E25
:10411000C96E8DEF20F0D6C1C9FF152A1200D7C194
:10412000C9FF152A1200D8C1C9FF152A1200D9C12A
:10413000C9FF152A1200C584152A1200FF0E156E3C
:104140001C9E12009E96C580152A1200E20EC96EB2
:10415000152A1200760EC96E152A1200C584152A7A
:104160001200FF0E156E1C9E1200C584142A156ADB
:1041700012009E96C580152A1200E20EC96E152AFD
:1041800012007B0EC96E152A120011AA04D0230E4C
:10419000C96E152A12001C0EC96E152A12009E96B1
:1041A000C580152A1200E20EC96E152A12007C0E77
:1041B000C96E152A1200E9D79E96C580152A1200ED
:1041C000E20EC96E152A12007D0EC96E152A120064
:1041D000DCD79E96C580152A1200E20EC96E152AFC
:1041E00012007E0EC96E152A1200CFD7C584152A7B
:1041F0001200FF0E156E1C9E12001550FF0AD8B457
:10420000BBEF21F0390EC86E800EC76E280EC66E49
:10421000000EC56E1450000AD8B416EF21F01450E9
:10422000010AD8B42AEF21F0BBEF21F01550000AA3
:10423000D8B468EF21F01550010AD8B46CEF21F022
:104240001550020AD8B476EF21F01550030AD8B4FD
:1042500079EF21F01550000AD8B47FEF21F0155006
:10426000010AD8B483EF21F01550020AD8B48DEFBB
:1042700021F01550030AD8B490EF21F01550040A2C
:10428000D8B496EF21F01550050AD8B499EF21F073
:104290001550060AD8B49FEF21F01550070AD8B47C
:1042A000A2EF21F01550080AD8B4A8EF21F015505C
:1042B000090AD8B4ABEF21F015500A0AD8B4B1EF0F
:1042C00021F015500B0AD8B4B4EF21F0BBEF21F068
:1042D0009E96C580BAEF21F016B004D04E0EC96E7E
:1042E000BAEF21F0500EC96EBAEF21F0C584BAEFD3
:1042F00021F0142AFF0E156E1280BBEF21F09E965E
:10430000C580BAEF21F016B004D04F0EC96EBAEFD7
:1043100021F0510EC96EBAEF21F0C586BAEF21F037
:10432000C9CF23F0C59AC588BAEF21F0C586BAEF88
:1043300021F0C9CF24F0C59AC588BAEF21F0C5860F
:10434000BAEF21F0C9CF25F0C59AC588BAEF21F0A0
:10435000C586BAEF21F0C9CF26F0C58AC588BAEF65
:1043600021F0C584BAEF21F0FF0E156E12861C9C59
:10437000BBEF21F0152A120012B012D012B213D0E6
:1043800012B414D012A6120007B01200129623C065
:1043900027F024C028F025C029F026C02AF01200FA
:1043A0001290128212001292128412000001155013
:0E43B000FF0A04E11294156AFDEC20F01200E1
:10BF0000E844F926000C160C2B0C3F0C520C640C68
:10BF1000760C860C960CA50CB30CC10CCF0CDC0C6B
:06BF2000E80CF40C000C1B
:00000001FF
